:020000000D28C9
:10000800DE0003088312A8000408A9000A08AA0051
:10001800C5288316FF23900083017F2900308A00BA
:100028000408840A82070034C034DE34A4348C34D3
:100038009A3489348134DC3480348834903483347D
:10004800E1348634A134B134EF34FD349034BB3418
:100058008C348934A334C134C0349B348034813423
:100068008234E034D434A834C434C634FD34DF34A4
:100078005A2110301721103039218519B615B619B3
:10008800851D62280230B5000330B400BA30B300D1
:10009800B30B4C28B40B4C28B50B4C2801308312F9
:1000A800B606B611361C5C281130172111303921DB
:1000B800361862281230172112303921361C682868
:1000C800B614831601176B28B61083160113831212
:1000D800361D41288B130D30B400FB30B300B30B31
:1000E8007328B40B7328782883123A0872213708CA
:1000F800B900BA0136118B010B170B168B17412863
:10010800A001A101A201A00A0319A10A05198728C3
:10011800A208031D982802302102BC3003192002CE
:10012800031898283908080000302102B53003194F
:100138002002A0010318A00AA10111302202031C09
:10014800AE28193022020318AD280310B80D200874
:10015800B8070310B70D2008B707A001A101051DB6
:10016800B328A20A21302202031C8728FF30B806D0
:1001780038083706031DC228370808000030B701C1
:10018800080001300B1E00398B1C00390038031D94
:10019800D428E828F2202008D2288420BA00E728AA
:1001A8000310B6180314003003180130A600A70185
:1001B8002708003A031DE7282608003A0319CE2825
:1001C800013A0319D12836158B102A088A00290804
:1001D800840028088300DE0E5E0E0900A301A40136
:1001E800A5010310A30DA40D031005190314003075
:1001F80003180130A3070318A40AFD30A20004293C
:100208000529A20B03290829092964008312A50AD4
:100218000E302502031CF628FF30A3062408A1008F
:100228002308A00008008312AC000510AE012C08BA
:10023800133E84001220AB002E0A24290310AB0CB5
:10024800FF3E031D22292B08AD002D1C2E298312E9
:10025800851430298312851005120516AE0A083058
:100268002E02031C1B2905140800AC000510AE0162
:100278002C08013E84001220AB002E0A45290310E9
:10028800AB0CFF3E031D43292B08AD002D1C4F2945
:100298008312851451298312851005120516AE0A9A
:1002A80008302E02031C3C29051408008B01831614
:1002B800850105150730831299001F1083169F11B9
:1002C8001F119F101F10831285010B108B110B1724
:1002D800831601178B100B168B170800AF00B2009E
:1002E800320E0F39B0003208B1000F30B1053008B6
:1002F800172131083929B601B701B801B901BA0186
:0403080083013C2809
:02400E00C43FAD
:00000001FF
